:100000000C9448060C943B330C9480060C948006A8
:100010000C9480060C9480060C9480060C94800648
:100020000C9480060C9480060C94C1290C947D29B4
:100030000C94142B0C9480060C9480060C9480066F
:100040000C9480060C9480060C9480060C94800618
:100050000C9480060C94F02A0C9480060C94800674
:100060000C9480060C9480060C9480060C948006F8
:100070000C9480060C9480060C9480060C948006E8
:100080000C9480060C9480060C9480060C948006D8
:100090000C9480060C9480060C9480060C948006C8
:1000A0000C9480060C9480060C9480060631FF099F
:1000B00074A1010975150026FF00952075088102BD
:1000C0000976150026FF00952075089102C00501EC
:1000D0000980A101850319012AB700150126B7007F
:1000E000950175108100C0050C0901A10185041955
:1000F000012AA002150126A002950175108100C0F9
:100100000660FF0961A1010962150026FF00952024
:10011000750881020963150026FF00952075089176
:1001200002C005010906A101050719E029E715002C
:100130002501950875018102950175088101050762
:10014000190029FF150026FF009506750881000596
:10015000081901290595057501910295017503910D
:1001600001C00000000000000000000000000000CE
:10017000000000000000000000000000000000007F
:100180000000000000007E0F00D4FFFFFFC700004A
:10019000007800000000000000002A2B280000006A
:1001A0000000000000000000000000000029000026
:1001B00000002C1E3420212224342627252E362D03
:1001C0003738271E1F202122232425263333362E9D
:1001D00037381F0405060708090A0B0C0D0E0F100F
:1001E0001112131415161718191A1B1C1D2F313054
:1001F000232D350405060708090A0B0C0D0E0F10F8
:100200001112131415161718191A1B1C1D2F313033
:10021000354C7267626C69676874206469736162E7
:100220006C65205B454550524F4D5D3A20726762C8
:100230006C696768745F636F6E6669672E656E616F
:10024000626C65203D2025750A007267626C6967E3
:10025000687420656E61626C65205B454550524F45
:100260004D5D3A207267626C696768745F636F6E98
:100270006669672E656E61626C65203D2025750A92
:10028000007267626C6967687420746F67676C6579
:10029000205B454550524F4D5D3A207267626C6954
:1002A0006768745F636F6E6669672E656E61626C06
:1002B00065203D2025750A0044454255473A206493
:1002C000697361626C65642E0A0044454255473A81
:1002D00020656E61626C65642E0A004F6E657368FE
:1002E0006F743A206163746976653A2025640A0068
:1002F0000A002530325820006B6579626F617264A4
:100300005F7265706F72743A200054617267657431
:1003100020636F6E6E65637465640D0A00546172CC
:1003200067657420646973636F6E6E65637465647A
:100330002C207468726F74746C696E6720636F6EC2
:100340006E656374696F6E20617474656D7074732B
:100350000D0A004661696C656420746F20657865DC
:10036000637574652025730A007267626C6967683B
:10037000745F636F6E6669672E7370656564203D98
:100380002025640A007267626C696768745F636F36
:100390006E6669672E76616C203D2025640A0072C6
:1003A00067626C696768745F636F6E6669672E73F6
:1003B0006174203D2025640A007267626C69676879
:1003C000745F636F6E6669672E687565203D2025D2
:1003D000640A007267686C696768745F636F6E6651
:1003E00069672E6D6F6465203D2025640A00726781
:1003F000626C696768745F636F6E6669672E656EAD
:1004000061626C65203D2025640A007267626C6938
:100410006768745F636F6E66696720454550524F29
:100420004D3A0A007267626C696768745F696E6949
:1004300074207267626C696768745F636F6E666967
:10044000672E6D6F6465203D20302E2057726974D1
:10045000652064656661756C742076616C75657382
:1004600020746F20454550524F4D2E0A007267622E
:100470006C696768745F696E6974206565636F6E27
:10048000666967206973206E6F7420656E61626CA7
:1004900065642E0A007267626C696768745F696ED2
:1004A0006974207374617274210A007267626C69E6
:1004B0006768745F696E69742063616C6C65642E33
:1004C0000A005B735D000A002530313662003A2075
:1004D0000025303258000A722F6320303132333415
:1004E00035363738394142434445460A007267621F
:1004F0006C6967687420616E696D6174696F6E20E4
:100500007469636B207265706F727420746F2073EE
:100510006C6176650A001E0F0500047F3F1F643280
:1005200014643214783C1E1E140A050A0025303269
:1005300058006C65645F7461736B3A200072676287
:100540006C6967687420656E61626C65205B4E4FF4
:10055000454550524F4D5D3A207267626C6967683D
:10056000745F636F6E6669672E656E61626C65208D
:100570003D2025750A007267626C69676874207394
:100580006574207370656564205B4E4F454550521D
:100590004F4D5D3A2025750A00000101010101015E
:1005A000010101020202020202020202030303032A
:1005B00003030303040404040404040505050505FA
:1005C00006060606060707070707080808080909B8
:1005D00009090A0A0A0B0B0B0C0C0C0D0D0D0E0E63
:1005E0000E0F0F0F101011111112121313141415F6
:1005F0001516161717181819191A1A1B1B1C1D1D6A
:100600001E1E1F20202122222324242526262728BF
:1006100029292A2B2C2D2D2E2F30313232333435EF
:10062000363738393A3B3C3D3E3F404142434445F2
:10063000464748494A4C4D4E4F50515354555658D1
:10064000595A5B5D5E5F616264656668696B6C6D7B
:100650006F7072737577787A7B7D7E8082838587F1
:10066000888A8C8E8F91939596989A9C9EA0A2A32F
:10067000A5A7A9ABADAFB1B3B5B7BABCBEC0C2C434
:10068000C6C9CBCDCFD1D4D6D8DBDDDFE2E4E7E9F4
:10069000EBEEF0F3F5F8FAFDFF7267626C696768DC
:1006A00074206D6F6465205B4E4F454550524F4D31
:1006B0005D3A2025750A007267626C69676874206C
:1006C0006D6F6465205B454550524F4D5D3A202566
:1006D000750A007267626C69676874206469736187
:1006E000626C65205B4E4F454550524F4D5D3A2040
:1006F0007267626C696768745F636F6E6669672EA4
:10070000656E61626C65203D2025750A0072676226
:100710006C696768742073657420687376205B4E1B
:100720004F454550524F4D5D3A2025752C25752C6F
:1007300025750A007267626C696768742073657456
:1007400020687376205B454550524F4D5D3A202519
:10075000752C25752C25750A007267626C696768AF
:1007600074207261696E626F77207365742068739C
:10077000763A2025642C25642C25642C25750A00E6
:10078000FFAA7F55400102030C0D0E0F000706055E
:10079000040B0A09087267626C69676874207469DF
:1007A0006D657220656E61626C65642E0A00726709
:1007B000626C696768742074696D6572206469731E
:1007C00061626C652E0A002223252628292A2C2DF9
:1007D0002F3032333536383A3B3D3E404243454771
:1007E000494A4C4E5051535557595A5C5E606264A9
:1007F0006668696B6D6F71737577797B7D7F8183B7
:100800008587898A8C8E90929496989A9C9E9FA1B7
:10081000A3A5A7A8AAACAEAFB1B3B4B6B8B9BBBCD8
:10082000BEBFC1C2C3C5C6C7C9CACBCCCDCED0D14D
:10083000D2D2D3D4D5D6D7D7D8D9D9DADADBDBDB45
:10084000DCDCDCDCDCDDDDDDDDDCDCDCDCDCDBDBE6
:10085000DBDADAD9D9D8D7D7D6D5D4D3D2D2D1D03A
:10086000CECDCCCBCAC9C7C6C5C3C2C1BFBEBCBB37
:10087000B9B8B6B4B3B1AFAEACAAA8A7A5A3A19FAF
:100880009E9C9A98969492908E8C8A898785838173
:100890007F7D7B79777573716F6D6B696866646254
:1008A000605E5C5A5957555351504E4C4A49474522
:1008B0004342403E3D3B3A3836353332302F2D2CC3
:1008C0002A2928262523224E004B00A900AA00C36E
:1008D0005CC45CAB00AC00C55CC65CC75CC85CCBF0
:1008E0005CCC5CC95CCA5C3A003B00165C1E001F15
:1008F0000020002100220023003C003D002B0014BA
:10090000001A0008001500170000003E003F0039E3
:100910000004001600070009000A00000040004122
:1009200000E10064001D001B0006001900050042E4
:10093000004300E000E200E30001512C002C000025
:100940000024002500260027002D002E004C002A40
:10095000004A001C0018000C00120013002F003089
:100960000031004D000B000D000E000F003300346D
:1009700000320028004B001100100036003700380C
:10098000000000E50052004E0001512C00E600E49A
:1009900000E7000000500051004F00010001001668
:1009A0005C3A003B003C003D003E003F000100017E
:1009B00000C25CC35C0100520001000100000001A4
:1009C00000010001000100500051004F0001000033
:1009D000000100010001000100010001000100010F
:1009E00000010001000100350201000100010001C9
:1009F0000001000000400041004200430044004567
:100A0000004C002A0001000100010001000100016A
:100A100000010001000100010001000100010001CE
:100A200000010001000100010001000100010001BE
:100A300000010001000000010001000100010001AF
:100A4000000100010001000000010001000100019F
:100A5000000100010001000100010001000100018E
:100A6000000100010001000100010001000100017E
:100A7000000000010001000100010001000100016F
:100A8000000100000001000100010001000100015F
:100A9000000100010001000100010001000100014E
:100AA000000100010001000000010001000100013F
:100AB000000100010001000100010001000100012E
:100AC000000100010001000100010001000100011E
:100AD000000100010001000100010001000100010E
:100AE00000010001000100010000000100010001FF
:100AF00000010001000100010001000000010001EF
:100B000000010001000100010001000100010001DD
:100B100000010001000100010001000100010001CD
:100B200000010001000000010001000100010001BE
:100B300000010001000100000001000100010001AE
:100B4000000100010001000100010001000100019D
:100B5000000100010001000100010000000100018E
:100B6000000100010001000100010001000100017D
:100B7000000100010001000100010001000100016D
:100B8000000100010001000100010001000100015D
:100B9000000100010001000100010001000000014E
:100BA000000100010001000100010001000100003E
:100BB000000100010001005B435D005B445D005BE0
:100BC000535D005B575D005B525D0009027B0004D2
:100BD0000100A0FA0904000001030101000921112C
:100BE00001000122400007058103080001090401FA
:100BF0000002030000000921110100012222000768
:100C000005820320000107050303200001090402F7
:100C10000001030000000921110100012232000738
:100C200005840320000109040300020300000009F9
:100C30002111010001222200070585032000010780
:100C4000050503200001120100020000000810CB7E
:100C50005743100401020001220351007500650092
:100C60006600720065006E0063007900200052008B
:100C7000650076002E002000340000000E034B00BB
:100C800065006500620069006F000000040309044C
:100C900011241FBECFEFDAE0DEBFCDBF04B603FEE6
:100CA00018C08091E7039091E803A091E903B09107
:100CB000EA038730904BA740B04B59F41092E703FA
:100CC0001092E8031092E9031092EA03E0E0F8E3DF
:100CD000099523E0AEE1B2E001C01D92A73EB20744
:100CE000E1F712E0A0E0B1E0EAE6FCE602C0059020
:100CF0000D92AE31B107D9F70E943B2B0C94083608
:100D00000C940000FF93EF93E0911E02F0911F02FC
:100D1000309709F00995EF91FF910895FC018591B5
:100D2000803011F0EFDFFBCF0895FF27E0E230E2E3
:100D300047FF0CC0419597FF09C0EDE260957095A3
:100D400080959095611D711D811D911D27FF02C029
:100D5000219530E350E2AA27660F771F881F991F5D
:100D6000AA1FA41710F0A41B63955A95A9F7AA30DF
:100D700008F0A95FA05DAF93F3956115710581053A
:100D8000910541F7ED3211F4EF93F395F21718F452
:100D90003F93F395FBCF8F91B5DFFA95E1F7089577
:100DA000E991F9918591803021F0853219F0AADF1F
:100DB000F9CF089520E0E89455915532C1F35033AE
:100DC00011F4689455915A3348F4505390F3220F1C
:100DD000022E220F220F200D250FF4CF0EF42195A5
:100DE00089919991533619F3533729F1533559F1B4
:100DF000BC0188279927E8945C3621F48991999160
:100E000068945591543639F446EF7EF077FF0DC063
:100E10008FEF9FEF0AC055374AE039F0583540E16F
:100E200021F0523642E009F00895FF93EF937DDF01
:100E3000EF91FF91B7CFFF93EF93FC018191803049
:100E4000B9F360DFFBCFFF93EF9368DFF1CFDF9360
:100E5000CF93CDB7DEB72596A3DFCF91DF9108956D
:100E6000E8EDF0E080818E7F80831092E2001092A6
:100E7000DA001092E100A0EEB0E08C9181608C93DA
:100E800080818F77808319BCA7EDB0E08C918E7F35
:100E90008C9380818F7E80831092CC030895209163
:100EA000E4003091E50095E6A9012091EC00822F45
:100EB000817020FF06C08091E80080FF06C080E0BE
:100EC00008952091E80022FD1AC08091D90388235B
:100ED00089F0853089F08091EB0085FD0FC020916D
:100EE000E4003091E50042175307F9F29150E1F622
:100EF00084E0089582E0089583E0089581E00895F4
:100F0000EF92FF920F931F93CF937C018B010E946E
:100F10004F07C82F811117C08091E80085FD0BC0D5
:100F20008091E8008E778093E8000E944F07882325
:100F300099F3C82F08C0F70181917F018093F100D8
:100F40000150110949F78C2FCF911F910F91FF90FC
:100F5000EF9008958091DB0387FF13C08091E80034
:100F600082FF06C08091E8008B778093E80004C080
:100F70008091D9038111F2CF08958091D9038823FC
:100F8000D9F38091E80080FFF8CF8091E8008E7758
:100F9000ECCF982F9093E900242F762F50E08917FB
:100FA00031F07091EC002091ED005091F00021FDA6
:100FB00007C09F5F973071F78093E90081E0089543
:100FC0003091EB003E7F3093EB003091ED003D7FA0
:100FD0003093ED003091EB0031603093EB00709373
:100FE000EC002093ED005093F0002091EE0027FDDF
:100FF000E0CF80E00895B0E0A0E0E1E0F8E00C94FC
:101000006134C8EDD0E088818F7E8883E7EDF0E021
:1010100080818160808384E082BF81E08093CC0303
:1010200088818E7F888302EE10E0F8011082109292
:10103000DA0081EEC82ED12CF601108288818F77DC
:10104000888388818068888388818F7D888319BCA4
:101050001092D9031092DA031092D8031092D7039A
:1010600090EEE92EF12CF70180818B7F80838881BF
:101070008160888342E060E080E00E94C907F60159
:1010800080818E7F8083F801808181608083808170
:1010900088608083F70180818E7F80838881806172
:1010A0008883CDB7DEB7E8E00C947D34FC018091F5
:1010B000E1039091E20386179707A0F0611571058F
:1010C00029F49091E8009E779093E80090E06115F4
:1010D000710551F4911108C08091E80082FF34C07D
:1010E00080E00895BC01F2CF8091D9038823C1F13B
:1010F0008530C1F18091E80083FD30C08091E80027
:1011000082FDEACF8091E80080FFE1CF8091F3007B
:101110002091F200382F6115710519F02830310542
:1011200058F091E02830310509F090E02091E80076
:101130002E772093E800CBCF81918093F10061500E
:1011400071092F5F3F4FE7CF8091D903882341F08A
:10115000853041F08091E80083FFBECF81E00895A3
:1011600082E0089583E00895089508950895809198
:10117000CE0308959C014FB7F8948091C2039091DB
:10118000C303A091C403B091C5034FBF821B930B4F
:1011900008952FB7F8946091C2037091C3038091B2
:1011A000C4039091C5032FBF08952FB7F894809181
:1011B000C2039091C303A091C403B091C5032FBF94
:1011C00008952091BF033091C0032817390771F0AB
:1011D0009093C0038093BF03E091BD03F091BE03E1
:1011E000309721F00084F185E02D09950895209134
:1011F000BB033091BC032817390771F09093BC03EF
:101200008093BB03E091BD03F091BE03309721F0C2
:101210000680F781E02D09950895FC01680F791F7C
:101220008FEF91E32191822728E030E087FF09C00A
:10123000880F892721503109C9F7E617F70791F779
:101240000895880FF7CFFA01811101C0FB010995BC
:1012500008958091B603982F9E7F29F48170826053
:101260008093B60308958635E8F381708465F8CFDE
:10127000AF92BF92DF92EF92FF920F931F93CF93A3
:10128000DF93082F162FE901E42FF0E0E756FA4F1D
:10129000611110C0E4915E2F4E2F4983E8835A8379
:1012A000DF91CF911F910F91FF90EF90DF90BF9052
:1012B000AF900895E62EF12C4491D42EE42FF0E067
:1012C00026E0829FC00111242FEF30E0B9010E9477
:1012D0009A34802F90E0880F991F55E5569FD001D2
:1012E000579FB00D11248A1B9B0B982F990F890FC4
:1012F0005901AE18BF08AE9ED001AF9EB00DBE9E84
:10130000B00D11245B2F189F80011124012F11278C
:101310005901A01AB10AAE9E8001AF9E100DBE9E6B
:10132000100D11245901A81AB108AE9CC001AF9C40
:10133000900DBE9C900D1124892F9927281B390BE5
:101340002E9FC0012F9F900D3E9F900D1124E92FDD
:1013500062307105A1F050F46115710509F49DCF5B
:101360006130710581F0EB2F512F97CF64307105FB
:1013700069F080F06630710509F48FCFF4CFE42F67
:101380004B2F592F8ACFE42F412F87CFEB2F542F8C
:10139000492F83CF4B2F5D2DE12F7FCFF894E82F7E
:1013A000E295EF70F0E031A1282F2F7081E090E0FE
:1013B00001C0880F2A95EAF7982F9095932391A35F
:1013C00092A1892B82A3789408959091EE0292FFC6
:1013D00006C0282F28712830F9F4877F846093FF96
:1013E00006C0282F28712831F1F4877E846120916E
:1013F000EF0220FF06C0382F38713830D9F4877FCC
:10140000816021FF06C0282F28712831D1F4877E02
:10141000816194FD877E0895282F24712430F9F688
:101420008B7F8860DCCF282F2471243101F78B7EDD
:101430008861DDCF382F3171313019F78E7F8860A8
:10144000E0CF282F2171213121F78E7E8861E1CFF5
:10145000CF93DF93EC0182389105B1F108F040C0E1
:101460008133910509F49DC048F58932910509F44D
:101470008DC08A9709F49CC0C11522E5D20708F0F7
:10148000BDC0C11531E5D30708F024C1C83ED10560
:1014900008F0A3C0C13ED10588F5C83AD10508F0CF
:1014A0008EC0C53AD10508F0F6C0C130D10531F182
:1014B000209721F1C430D10508F545C08533910549
:1014C00009F45FC0C997C1F68091EE02837009F0FC
:1014D00036C18091EF0283FF11C0C9E2D0E00EC097
:1014E000833E910599F170F4803E910501F1823EB1
:1014F000910511F68091EE0282FD21C0CE01DF91AF
:10150000CF910895863E910561F1873E910571F175
:10151000843E910509F0B0CF8091EF0281FFEECFBC
:101520008091EE02C7EED0E084FD0DC0E7CF809140
:10153000EE0280FD33C09091EF0290FFDFCFC3EE4B
:10154000D0E084FFDBCFD0E0C0E0D8CF8091EE02C6
:1015500082FDF2C09091EF0290FDF1C084FFCECFEA
:10156000F2CF8091EE0283FDDDCFC8CF8091EE02F5
:1015700083FDE8C09091EF0291FFF0CFC4EED0E080
:10158000BDCF8091EE0285FFB9CFA7CF8091EE024B
:1015900085FDDBC08091EF0283FFB0CFC9E3D0E0CF
:1015A000ADCF8091EE0286FFA9CFCAE2D0E0A6CFF0
:1015B0008091EE0286FFA2CFC1E3D0E09FCFCF3B68
:1015C000D10508F6C85AD0E0CC0FDD1FC156DE4F5A
:1015D0000990D881C02DD46491CFC11540E5D407BE
:1015E00008F064C0C11580E4D80708F05CC0CE01E3
:1015F0009A9581159F4108F481CFA5CFC11536E595
:10160000D30718F5C11545E5D40708F07CC0C1150E
:1016100084E5D80708F072C09E01237033279C2F01
:1016200096959695C115D34508F459C0C1E0D0E010
:1016300002C0CC0FDD1F2A95E2F730E2939FC00174
:101640001124C82BD92BDA6859CFC1158AE5D807E0
:1016500078F4C11529E5D20708F060C0C11538E556
:10166000D30708F470CFDC2FCC27C06FD06A46CFE9
:10167000CE0190568115904208F065CF8D2F8F7165
:101680000E94E50990E0982F882788279F719C0188
:101690002C2BE90141C0C55AD0E0C456DE4FC881A9
:1016A000D0E0D0642BCFDF70D06A28CFCE0183701A
:1016B000992721E030E002C0220F331F8A95E2F71C
:1016C000C695C69580E2C89FE0011124C22BD32B9A
:1016D000DD6814CFDC2FCC27C16FD06A0FCFC1E0FB
:1016E000D0E002C0CC0FDD1F2A95E2F720E2929FE6
:1016F000C0011124C82BD92BDC6800CFDC2FCC27EC
:10170000C46FD06AFBCE8C2F0E94E509C82FD0E0B1
:10171000DC2FCC27CC27DF71D062F0CE8C2F8F70DE
:101720000E94E50934E0D695C7953A95E1F7CF7068
:101730009C2FEC01D069E2CEC2EED0E0DFCEC0EE4D
:10174000D0E0DCCEC6EED0E0D9CEC5E3D0E0D6CE38
:101750000E94C9080895809193028111109293020A
:101760000895809590919202982390939202089503
:10177000E2E2F2E09191891303C0DF0111971C921C
:1017800092E0E832F907B1F70895A2E2B2E0EFEF94
:1017900090E02D91821751F0EF3F19F4211101C013
:1017A000E92F9F5F9630A9F7EF3F09F408950E2EB9
:1017B000000CFF0BE05EFD4F82830895809187024D
:1017C00090915602981301C008958F5F8770FACFE9
:1017D000A82FA77023E0969587952A95E1F7FC013D
:1017E000EE0FFF1FE80FF91FE60FF71F50E040E074
:1017F00080E0219130E00A2E02C0369527950A94A8
:10180000E2F721703327042E01C0220F0A94EAF771
:10181000822B4F5F5F4F4330510559F70895292FB1
:101820009A3068F4893090F490E06CE272E039E02C
:10183000239F800D911D11240E94E80B08952C5FB9
:10184000223020F469E272E090E0F6CF80E0089563
:10185000262F277091E001C0990F2A95EAF723E01F
:10186000769567952A95E1F7FB01EE0FFF1FE60FCE
:10187000F71FE40FF51F50E040E0682F70E0819102
:10188000DF0111979B01042E02C0369527950A941B
:10189000E2F7217021952827292328272C934F5FD1
:1018A0005F4F4330510559F70895282F862F9A30FE
:1018B00070F4293058F4622F70E029E0929F600D97
:1018C000711D11244CE252E00E94280C08959C5F87
:1018D0009230E0F7622F70E049E252E0F5CF829556
:1018E00090E09C01220F331F220F331F2C7C959513
:1018F0008795959587958373282B30E0C901880FCC
:10190000991F8A7A359527952575822B08959FB75B
:10191000F8941092CA039FBF9091D903943009F0B4
:1019200048C02091E9002F703091EC00932F917006
:1019300030FD90E8922B25E02093E9002091EB0008
:1019400020FF34C02091EE0027FF30C02091C90352
:10195000222321F02091E80025FF28C01092C9031E
:1019600026E03091E80035FF14C08093F1008091AB
:10197000E80085FD27C08091E80080FFFCCF8091C2
:10198000E8008E778093E8009F709093E90080E0F4
:1019900008953091D903343049F43091EB0035FD8E
:1019A00005C0215041F481E08093C9039F7090935A
:1019B000E9008FEF0895EFE9FFE03197F1F700C0FC
:1019C0000000CFCF8FB7F89421E02093CA038FBFD8
:1019D000DBCF8093C6037093C8036093C7038091E5
:1019E000D9038430F9F48093E9008FEF9091E800F7
:1019F000815095FD06C095ED9A95F1F70000811193
:101A0000F5CF8091E80085FF0DC050E040E063E035
:101A100070E086EC93E00E9480078091E8008E776A
:101A20008093E8000895BC0184E00E94E90C0895C9
:101A3000BC0183E00E94E90C0895CF93DF93EC0191
:101A400081E08093E9008FEF9091E800815095FD4F
:101A500006C095ED9A95F1F700008111F5CF8091C0
:101A6000E80085FF14C050E040E068E070E0CE017F
:101A70000E9480078091E8008E778093E80088E0DC
:101A8000FE01AFECB3E001900D928A95E1F7DF9192
:101A9000CF91089581E08093E00080E28093D800A8
:101AA0001092C9008FE19EE40197F1F700C0000099
:101AB00087E090EBDC018093E7039093E803A09329
:101AC000E903B093EA0388E19CE00FB6F894A89587
:101AD000809360000FBE90936000FFCFCF92DF92A3
:101AE000EF920F931F93CF93DF93CDB7DEB7E097BD
:101AF0000FB6F894DEBF0FBECDBF6091600180913C
:101B0000B60380FF4BC0E5E8F7E09E012F5F3F4F33
:101B10008E010F5C1F4FC901A4914A2F50E0DA01DA
:101B2000AA0FBB1FA40FB51FAA5CBC4FCD90DD90C0
:101B3000EC90D901CD92DD92ED929D013196A017E6
:101B4000B10751F720915F0143E0249F800D911D63
:101B500011246E9A2EB12F7B3EB130645FB7F8949A
:101B6000FC01649FE00DF11D1124BF01861797074A
:101B700041F55FBFEFE5F4E03197F1F700C00000F9
:101B8000E0960FB6F894DEBF0FBECDBFDF91CF91C8
:101B90001F910F91EF90DF90CF9008958091610198
:101BA0009091620123E0829FF0011124EA5CFC4FD6
:101BB000891708F0A8CF1182108212828F5F3396A6
:101BC000F7CFDC014D91CD01E8E03EB9000000C047
:101BD00047FF2EB9440F000000C000C000C02EB95E
:101BE00000C0EA9591F7C2CF0F931F93CF93DF9375
:101BF000EC0110E000E0909163019017110609F0EC
:101C00006CF40E946E0D8C8190E001968170992792
:101C10008C83DF91CF911F910F91089520916101E5
:101C2000A801420F511D9A01220F331F240F351FA7
:101C30002A5C3C4F4C816091B8038091B703969524
:101C40009017110651F04CF0442349F04091B9032C
:101C50000E9438090F5F1F4FCECF4423B9F340E0F5
:101C6000F7CFB0E0A0E0E7E3FEE00C945D34EC01D8
:101C70004C81042F10E09801D8010E94F9359B0196
:101C8000AC010E94C4354B015C01E0E2F0E0E01BD6
:101C9000F10BA5E5B0E0AC019B010E94C4356B01DE
:101CA0007C019F01DF010E94CF349B01AC010E94A7
:101CB000CF359B01AC01280D391D4A1D5B1DC701A5
:101CC000B6010E94D735F22E822F90E039E23F15FF
:101CD00020F143E0249F9001112435952795122F80
:101CE000109500E085E5E82EEF1880916301081754
:101CF00018F10E946E0D9C8181E0992319F09032B9
:101D000019F48FEF80935E0180915E01890F8C83BF
:101D1000CDB7DEB7ECE00C94793425E530E0B901BD
:101D2000681B790B9B01220F331F260F371F37FFCC
:101D3000D4CF2F5F3F4FD1CF8E2D01FD8F2D20911E
:101D40006101622F600F7727771F9B01220F331FDE
:101D5000260F371F2A5C3C4F412F6091B8030E9429
:101D600038090F5FC2CFEF92FF920F931F93CF936B
:101D7000DF93EC018C81811109C081E08C8310928A
:101D8000340392E090935D0180935C018091610146
:101D90009091620123E0829FF0011124EA5CFC4FE4
:101DA000891758F110E003E060916301161758F1AC
:101DB0000E946E0D80915C0120913403280F2093C6
:101DC000340390915D01980F90935D01191654F4BE
:101DD000022E000C330B409163014150550B241728
:101DE000350734F0819580935C01813009F41C82C1
:101DF000CDB7DEB7E6E00C947F34118210821282F8
:101E00008F5F3396CDCFE12EF12C70E0C7010E9499
:101E1000AE3420916101820F482F50E020913403AD
:101E2000022E000C330BE216F306BCF020915D018C
:101E3000022E000C330B2E153F057CF0809F900185
:101E400011242A5C3C4F4091B9036091B803809102
:101E5000B7030E9438091F5FA7CFFA01EE0FFF1FDB
:101E6000E40FF51FEA5CFC4F118210821282F3CF5F
:101E7000B0E0A0E0EEE3FFE00C945E34EC018A8178
:101E8000BB24BA9480FD02C0BB24B394A09063012C
:101E90008C81811109C081E0B8121EC08FEF8A0DBC
:101EA0008093330381E08C83F12CE12CEA14B8F0A9
:101EB0000E946E0D8091330391E0B91254C08111DC
:101EC0004DC0809163018150809333031C82CDB754
:101ED000DEB7EBE00C947A3410923303E3CF009139
:101EE00061010E0D1F2D111DC801880F991F080FCC
:101EF000191F0A5C1C4FF80111821082128234E013
:101F0000C32ED12C912C80913303890D813114F192
:101F10008F70082E000C990B8E159F0591F48091FF
:101F2000B9038C9DA0018D9D500D112455954795A9
:101F30005595479598016091B8038091B7030E9429
:101F400038099B0CF1E0CF1AD108E9F68FEFE81AB7
:101F5000F80AACCF87FFDDCF8A0DDBCF81508093AD
:101F60003303BC82B4CF90E001966091630170E0CE
:101F70000E94AE34809333038C83A9CFEF92FF92FB
:101F80001F93CF93DF93EC0110E0EE24EA94F12C41
:101F900060916301161770F00E946E0D9A818C811A
:101FA00090FF27C08F5F8C83DF91CF911F91FF90AF
:101FB000EF90089520916101422F410F5527551F41
:101FC000CA019A01220F331F280F391F2A5C3C4F88
:101FD00070E0C7010E94AE34962F8C814091B90306
:101FE0006091B803199F800D11240E9438091F5F6A
:101FF000CFCF8150D8CF9091B60390FF0EC0909173
:1020000061012091620133E0939FF0011124EA5CA9
:10201000FC4F921718F00E946E0D08958183608323
:1020200042839F5F3396F5CFA3E0B0E0EAE1F0E1B1
:102030000C9465348C018091350381110AC09E0196
:102040002F5F3F4F4FEF6FEF0E9438098A818093D7
:102050003503F8016481613069F08091350340E017
:10206000662361F040E0623011F44091350380E076
:1020700060E004C06091350340E080E00E94FB0F07
:10208000F801848190E0019663E070E00E94AE3434
:1020900084832396E4E00C948134A3E0B0E0E3E58C
:1020A000F0E10C9467349091B60390FF0AC09E0152
:1020B0002F5F3F4F0E9438094B8169818A810E94BE
:1020C000FB0F2396E2E00C948334CF93DF93EC0173
:1020D000E6EBF3E0438162818C810E944D108C819C
:1020E0008F5F8C83DF91CF910895CF93DF93EC01C5
:1020F000EC81F0E0E953F84F4491E6EBF3E06281C4
:1021000081810E944D108C818F5F8C83DF91CF91F4
:10211000089580919F02811110C08091D800806144
:102120008093D8008AE18A95F1F700C08091D900A8
:1021300080FF0AC081E080939F0281E090919F021E
:10214000913009F080E0089582E080939F020E9420
:1021500030071092D903F1CF0E948910882359F0DB
:10216000E091BD03F091BE03309729F00190F0811A
:10217000E02D0995089580E008950F931F930E9424
:102180008910882329F00E94C9081F910F91089592
:102190000E94C9080091D4021091D5022091D60264
:1021A0003091D702600F711F821F931FEECF0E94E4
:1021B0008910882319F00E94D50808950E94BD1047
:1021C000CB010895CF93DF93C7E1D3E060E0CE0168
:1021D0000E9471352196C11584E0D807B9F7DF91C7
:1021E000CF9108950F931F93CF93DF93142F022F56
:1021F000843020F5623010F598E0899FE0011124C9
:1022000084E0689FB0011124C60FD71FC950DD4F6D
:1022100082E090E0442311F090E080E0632F8C0F87
:102220009D1F0E94713583E090E0112311F081E041
:1022300090E0602F8C0F9D1F0E947135DF91CF9130
:102240001F910F9108951F93CF93DF93122F843026
:10225000E0F46A30D0F44930C0F4C42FD0E0CC0FA1
:10226000DD1F92E1699FC00DD11D112494EB899F60
:10227000C00DD11D1124632FCE0187960E947135A8
:10228000612FCE0188960E947135DF91CF911F9109
:102290000895B0E0A0E0EFE4F1E10C945D3487EC48
:1022A000E82E88E0F82E07EE18E0C0E05801D0E0F4
:1022B00015C0F401259134914D2D6D2F8C2F0E9466
:1022C000231182E0880E911CD39489E0D812F1CFBB
:1022D00082E1A80EB11CDF5FDA3019F04501D12C84
:1022E000E8CF6701D0E0F6012591349141E06D2FF0
:1022F0008C2F0E94F210F60132962591349140E025
:102300006D2F8C2F0E94F21084E0C80ED11CD130AA
:1023100071F488E0E80EF11CCF5F0C541F4FC430FD
:1023200009F0C4CFCDB7DEB7ECE00C947934D1E03E
:10233000DACFCF93C82F6FEF811162E283E290E092
:102340000E9471356FEFC11163E084E290E00E945A
:1023500071356FEFC11160E185E290E00E94713547
:10236000CF91089580E00E94991160E086E290E0AC
:102370000E9471350E9449110E94E21081E00E9482
:1023800099110895FF920F931F93CF93DF93F42E2B
:10239000843070F5623060F528E0829F800111245E
:1023A00034E0639FB0011124060F171F09501D4F21
:1023B00082E090E0442311F090E080E0800F911FD4
:1023C0000E945D35C82FD0E0DC2FCC2783E090E061
:1023D000FF2011F081E090E0800F911F0E945D3599
:1023E0009E01282BC901CDB7DEB7E5E00C948034FF
:1023F00090E080E0F8CF0F931F93CF93DF9384306A
:1024000030F56A3020F5493010F5C42FD0E0CC0FFC
:10241000DD1F22E1629FC00DD11D112434EB839F8B
:10242000C00DD11D1124CE0187960E945D35082F65
:1024300010E0102F0027CE0188960E945D3598018C
:10244000282BC901DF91CF911F910F91089590E042
:1024500080E0F8CF843070F47A3038F4693050F48A
:10246000462F672F0E94FB1108957D3F31F441E014
:10247000623040F090E080E008957C3FD9F7623010
:10248000C8F740E00E94C2110895CF92DF92FF92F8
:102490000F931F93CF93DF936C010091E60380911C
:1024A0009402082BC7E0D0E010E0FC2EC8010C2EEF
:1024B00002C0959587950A94E2F780FD0CC021979C
:1024C000A0F7F12C8F2DDF91CF911F910F91FF90ED
:1024D000DF90CF900895B6018C2F0E942A120E949F
:1024E000280A019761F3EECFCF93DF93EC010E94AE
:1024F0004512BE010E942A120E94280ADF91CF9144
:102500000895FC0183819481892B29F08081918138
:1025100089238F3F51F480E00895843FE1F717C08D
:10252000883EA8F0813FB9F712C0808191810E9456
:10253000741292959F70963099F358F4925F9F7041
:10254000923048F7803F19F040F7883E20F781E04D
:1025500008959A5FF4CF83E290E00E945D35823265
:1025600089F484E290E00E945D35833059F485E27D
:1025700090E00E945D3591E0803109F090E0892F74
:102580008170089580E0FCCFCF9384E090E00E94BA
:102590005D35C82F82E290E00E945D35982F8C2F28
:1025A000CF910895B0E0A0E0E8EDF2E10C94593449
:1025B000FC016280448081E08483E7ECF7E0749062
:1025C000E6E4F8E0E491812C75E0972EF2E0CF2E5E
:1025D000DD24D394AA24AA94B12C55245A94E71943
:1025E0000E2F10E080916301881638F00E946E0D66
:1025F000CDB7DEB7E0E10C947534E82CF12C82E025
:10260000861568F09E9CF0019F9CF00D1124EA59FC
:10261000FC4F8091B70380838091B8038183411080
:1026200023C09E9CF0019F9CF00D1124EA59FC4FA1
:102630001382128220916101C701820F911D9C01BA
:10264000220F331F280F391F2A5C3C4F9E9CF0013C
:102650009F9CF00D1124EA59FC4F428161818081D9
:102660000E9438098394BECF9E9CE0019F9CD00DB0
:102670001124CA59DC4F8B818823E9F081508B8368
:10268000859DC00111246C8170E00E949A34FB0189
:10269000FF27E953F84F8491E82FE719E59DC00122
:1026A0001124B8010E949A348091B903689FB00147
:1026B00011247A83BFCF0E942A352091B903269531
:1026C00021582C9DA0012D9D500D1124452F5527DB
:1026D000841795070CF0AECF82E0861588F40E942F
:1026E0002A35B5010E94AE3488830E942A35209194
:1026F000B8032695622F70E00E94AE34280F29831C
:102700009E9CF0019F9CF00D1124EA59FC4F12820F
:102710008091B903893C58F088EC9E9CF0019F9C05
:10272000F00D1124EA59FC4F8483838383CF8431D5
:10273000A0F784E1F2CF10923103809132038460DC
:102740008093320380912F0380FF08C08EEA97E0C8
:102750009F938F930E9427070F900F900895809169
:10276000B6038E7F8093B60380912F0380FF0CC049
:102770001F921F9283ED96E09F938F930E942707ED
:102780000F900F900F900F900E949B138091320337
:102790008160809332032FEF80E792E021508040E8
:1027A0009040E1F700C000000E946E0D0895B0E077
:1027B000A0E0EDEDF3E10C945C347C015B01842E30
:1027C000752E69018091A00201E010E08A3010F4BA
:1027D0000AE010E0C1E0D0E0B501C701F6010995BB
:1027E000982E811114C021960C171D07B4F4809106
:1027F0002F0380FF0CC07F928F9283E593E09F931D
:102800008F930E9427070F900F900F900F90892DA4
:10281000CDB7DEB7EDE00C947834CC9F9001CD9F1E
:10282000300D300D112490E080E045E34A95F1F73A
:102830000000019628173907C1F7CECF6091B60383
:10284000669570E04BE050E081E591E00E943A35FA
:10285000892B19F481E0809331030E94D710909363
:102860002A0380932903809132038460809332038A
:1028700080912F0380FF08C085E997E09F938F9395
:102880000E9427070F900F900895CF92DF92EF924A
:10289000FF926B017C010E942909B701A60188E023
:1028A00090E00E948335FF90EF90DF90CF900895E5
:1028B000A3E0B0E0EEE5F4E10C945A34082FE62EE4
:1028C000F42EC22E9091B60390FF57C0E92FE695E3
:1028D000AE2FB0E0A152BE4F8C91809330039E7F0B
:1028E000923009F04EC09E012F5F3F4F802F0E9413
:1028F00038094B8169818A810E94FB0F8091B7035F
:10290000801308C08091B8038E1104C08091B90370
:102910008F1529F0809132038260809332030093F7
:10292000B703E092B803F092B903CC2009F486C053
:102930006091B6037091B7038091B8039091B90389
:102940000E94451480912F0380FF17C08091B90326
:102950001F928F938091B8031F928F938091B7033A
:102960001F928F9384E397E09F938F930E94270792
:102970000FB6F894DEBF0FBECDBF2396EFE00C94E8
:102980007634823019F4F090B903B8CF863019F458
:102990000091B703B3CF8930D9F3893109F0AECFB5
:1029A000E9518E2F8170782E8E2F80958170D82ED0
:1029B000E695F0E0E058F84F1491612C99E5A92EC6
:1029C00097E0B92E60916301661618F00E946E0DB3
:1029D00095CF619EC001112470E00E949A34502E60
:1029E00071102AC0560E862C912C80912F0380FFE7
:1029F00011C01F921F931F92DF921F925F921F922E
:102A00006F92BF92AF920E9427070FB6F894DEBF75
:102A10000FBECDBF20916101820E911C9401220F47
:102A2000331F280D391D2A5C3C4F4F2D6E2D852DEF
:102A30000E9438096394C6CF561AD5CF80912F03D0
:102A400080FF9BCF1F92FF921F92EF921F920F93D6
:102A50008DE097E089CFE6EBF3E0438121E1421B73
:102A600008F440E021E0628181810E9458140895B9
:102A7000E6EBF3E0438121E1420F08F44FEF21E060
:102A8000628181810E9458140895E6EBF3E062812F
:102A900021E1621B08F460E021E0438181810E9412
:102AA00058140895E6EBF3E0628121E1620F08F427
:102AB0006FEF21E0438181810E9458140895E6EB75
:102AC000F3E0818121E04381628188500E945814A3
:102AD0000895E6EBF3E0818121E043816281885F24
:102AE0000E94581408958091BA03882319F08150E8
:102AF0008093BA036091B6037091B7038091B803D5
:102B00009091B9030E94451408958091BA038330CF
:102B100018F48F5F8093BA036091B6037091B70386
:102B20008091B8039091B9030E9445140895909143
:102B3000B60390FF45C09170811143C0926090939D
:102B4000B60380913203816080933203662309F4D7
:102B50003FC06091B6037091B7038091B803909124
:102B6000B9030E94451480912F0380FF0FC080910C
:102B7000B60386951F928F9387EB96E09F938F9372
:102B80000E9427070F900F900F900F906091B6034F
:102B9000669570E04BE050E081E591E00E943A35A7
:102BA000892B11F10E949B1381E080932C0320E07C
:102BB0004091B9036091B8038091B7030E94581403
:102BC00008958B3210F09465BACF880F982BB7CF49
:102BD00080912F0380FFDACF8091B60386951F92F4
:102BE0008F9389E996E0CACF0E941E14DDCF8091B1
:102BF000B6038695815009F48AE261E00E94971538
:102C000008958091B60386958F5F8B3208F081E03E
:102C100061E00E94971508959091B60390FF08C057
:102C20009695981728F0961718F40E9401160895A3
:102C300061E00E9497150895E6EBF3E087E1808359
:102C400011828FEF828383831482A0E3B3E0129614
:102C50008C911297836012968C936081718182812E
:102C600093810E944514089568EE7EEF90E080E025
:102C70000E948F3560E082E090E00E94713560E054
:102C800083E090E00E9471351092940260E084E04D
:102C900090E00E94713564E082E290E00E9471351C
:102CA00060E085E090E00E94713560E086E090E0B1
:102CB0000E9471356FEF87E090E00E94713540E02F
:102CC00050E0BA0188E090E00E94833560E08DE03A
:102CD00090E00E94713540E050E0BA0188E190E058
:102CE0000E94833560E087E190E00E94713540E00A
:102CF00050E0BA018CE190E00E94833570E060E022
:102D000080E290E00E948F3540E050E0BA0188E117
:102D100090E00E94833580E00E9499110E94B211D8
:102D200040E050E0BA018FE090E00E94833540E03F
:102D300050E0BA0183E190E00E9483350895A8E055
:102D4000B0E0E5EAF6E10C94673485E0E6EBF3E009
:102D5000DE01119601900D928A95E1F78091300382
:102D600090913103A09132038E839F83A887288599
:102D70004091D0025091D1026091D2027091D30261
:102D80003FB7F8948091C2039091C303A091C4030C
:102D9000B091C5033FBF841B950BA60BB70B8436C0
:102DA0009105A105B10510F4222319F180912D019F
:102DB00090912E0189549D4F40912C0150E0493053
:102DC000510510F048E050E0BE016F5F7F4F0E9458
:102DD000543585E090E00E94E133882369F00E9439
:102DE000C9086093D0027093D1028093D20290936D
:102DF000D3021092320381E02896E2E00C948334EF
:102E0000A4E0B0E0E6E0F7E10C9466344091B30250
:102E10005091B4026091B5027091B6022FB7F89448
:102E20008091C2039091C303A091C403B091C503E4
:102E30002FBF841B950BA60BB70B11E084369105B1
:102E4000A105B10570F10E94BD106E5F7F4F8F4FDD
:102E50009F4F69837A838B839C8380912501909116
:102E6000260189549D4F4091240150E04530510581
:102E700010F044E050E0BE016F5F7F4F0E94543578
:102E800084E090E00E94E133182F882351F00E94E3
:102E9000C9086093B3027093B4028093B502909313
:102EA000B602812F2496E3E00C9482344F925F9215
:102EB0007F928F929F92AF92BF92CF92DF92EF92CA
:102EC000FF920F931F93CF93DF930F92CDB7DEB78F
:102ED000C62E4A015901482E880F5508C2010E948A
:102EE000E133782E882309F480C0C20133E0880FD3
:102EF000991F3A95E1F7FC01EC5FFE4F438150E0EA
:102F00004115510511F041E050E08C5F9E4FFC01EE
:102F10006481758169547D4FCE0101960E945435BC
:102F2000F40140815181628173812FB7F8948091BF
:102F3000C2039091C303A091C403B091C5032FBFF6
:102F4000841B950BA60BB70B84369105A105B10523
:102F500040F4B701C8010E940D099981891709F44D
:102F600044C00C2C000CDD08C6010E94E133782E11
:102F7000811113C0712C872D0F90DF91CF911F917C
:102F80000F91FF90EF90DF90CF90BF90AF909F9008
:102F90008F907F905F904F900895C60123E0880F37
:102FA000991F2A95E1F7FC01EC5FFE4F438150E049
:102FB000E416F50608F4A7018C5F9E4FFC016481BE
:102FC000758169547D4FC5010E945435B701C80110
:102FD0000E940D0999818913CDCF0E94C908F4017F
:102FE0006083718382839383C6CFA701B801C50133
:102FF0000E945435C0CFAAE0B0E0E1E0F8E10C94C3
:1030000061346B018AE0E82EF12C08EB12E09E019E
:103010002F5F3F4F4BEA52E061E080E00E9456177D
:10302000882349F09AE0FE013196A1EAB2E00190CE
:103030000D929A95E1F79AE0E1EAF2E0D60101906B
:103040000D929A95E1F72A96E8E00C947D34AEE172
:10305000B0E0EDE2F8E10C9459348E010F5F1F4FA0
:1030600084E1D8011D928A95E9F76DE3E62E61E0CF
:10307000F62E680172E4472E71E0572E66246394A1
:10308000712CFDE38F2EF1E09F2EF70181917F01DE
:103090008F3F09F445C0F894E82FE295EF70F0E017
:1030A00021A18F70A30102C0440F551F8A95E2F73A
:1030B000CA01922F982B91A392A18095892382A374
:1030C000789400C0E4E3F1E021E030E0B12CA12CE1
:1030D00041914F3F09F46DC0A42FA295AF70B0E0AD
:1030E00090968C9190E04F7002C0959587954A9587
:1030F000E2F780FD5EC0C901A82AB92A220F331F5A
:103100008E169F0629F7F701319780818F3F11F0C6
:103110000E94CE0950EA5A95F1F7D601AD92BC92C1
:10312000B2E0CB0ED11C4E145F0409F0AECF44E1E7
:1031300050E0B80188ED92E00E944735009741F0D9
:1031400024E1F801A8EDB2E001900D922A95E1F793
:103150000091ED02892B81F181E0809397020E941A
:10316000D508909396028093950280919502909154
:1031700096020E94BA08059718F110E0000F111F7F
:103180000B5E1C4F4AE050E068ED72E0C8010E94FF
:103190004735C12C892B51F08AE0E8EDF2E0D801E7
:1031A00001900D928A95E1F7CC24C3941092970276
:1031B00008C090E080E0A0CF809197028111D5CF28
:1031C000C12C0E948910D82EE091ED02AE014B5E19
:1031D0005F4F7A01882309F4A1C08AE0DA011D92C9
:1031E0008A95E9F70E2F10E0000F111F0B5E1C4FA0
:1031F000B090A002B9E0BB1508F44AC02BEF37E14C
:1032000043E751E0B701C8010E94D713882309F4AE
:1032100063C028E139E240E851E0B701C8010E94EB
:10322000D713882309F458C020E037E148E851E07B
:10323000B701C8010E94D713882309F44DC02FE9B4
:1032400036E143E951E0B701C8010E94D713882352
:1032500009F442C0F9E0FB1508F457C01092A0022F
:103260008091EC0290E0880F991F4AE050E0B7018E
:103270008B5E9C4F0E94473521E020939E02892B54
:10328000E1F4D12C8D2D8C296E96E0E10C947534EF
:1032900080919802909199020E94BA08843F9140CF
:1032A00008F0ACCF80919E02882359F38AE0D701C1
:1032B0001D928A95E9F710929E02A091EC02B0E06F
:1032C000AA0FBB1FAB5EBC4F8AE0FE017596019052
:1032D0000D928A95E1F7D6CF8091A0028F3F31F011
:1032E0008F5F8093A0028A3008F4BACF0E94D5087D
:1032F000909399028093980280912F0380FFD2CF00
:103300008DE193E00E948E06CDCF80912F0380FF48
:10331000A5CF8AE093E00E948E06A0CFF0E0EE0FEA
:10332000FF1FEB5EFC4F8AE0A8EBB2E001900D922C
:103330008A95E1F76AE070E088EB92E00E940D095F
:103340008093B7024091110350E06091100370E048
:10335000645F7C4FC7010E9454358D898093C302FE
:1033600061E070E0C7010E940D098093C202809065
:10337000C4029090C502A090C602B090C70280918E
:103380009A0290919B02A0919C02B0919D02881696
:103390009906AA06BB06D1F080929A0290929B02EF
:1033A000A0929C02B0929D020E94891081110EC0D1
:1033B0000E94C908861A970AA80AB90A8092D402FC
:1033C0009092D502A092D602B092D7028091CF02FD
:1033D000882309F457CF80FF0DC08091C80280FF79
:1033E0002AC09091B60391609093B60360E08695F1
:1033F0000E9497158091CF0281FF09C020E0409183
:10340000CB026091CA028091C9020E945814809137
:10341000CF0282FF06C08091CE02882379F00E94FD
:103420001E148091CF0283FF03C081E080932C03A0
:103430001092CF0227CF0E94AF13DCCF0E949B13C4
:10344000F0CF0F931F93CF93DF93809192029091CF
:103450009102892B8093200290919302992391F0FD
:10346000892B8093200220E082E292E0FC013191DE
:10347000CF0131112F5FF2E088329F07B9F7211198
:103480000E94AB0B48E050E069E872E080E292E015
:103490000E944735892B09F441C088E0E0E2F2E060
:1034A000A9E8B2E001900D928A95E1F7E091BD03A1
:1034B000F091BE03309791F10280F381E02D80E21C
:1034C00092E0099580912F0382FF28C080FF04C0FD
:1034D00088EF92E00E948E06D0E0C0E002EF12E09A
:1034E00080912F0380FF0EC0FE01E05EFD4F8081C2
:1034F0001F928F931F930F930E9427070F900F9097
:103500000F900F902196C830D10551F780912F036D
:1035100080FF04C080EF92E00E948E06DF91CF9181
:103520001F910F91089590E080E00E94F70890E0CD
:1035300080E00E94E108109291020E94211A0895F1
:103540008093E6030E94931A08958091E603982FD2
:103550009670963021F488600E94A01A0895877FA3
:10356000FBCF21E030E001C0220F8A95EAF72095D9
:103570008091E60382230E94A01A08959091880208
:103580008095892380938802282F277091F4282F13
:10359000082E000C330B9217130659F09091EF028E
:1035A00092FF07C08595859585950E94B11A109266
:1035B00088020895CF93DF93D82FC091EF02C2FB0A
:1035C000882780F98D1711F1D0FBC2F9C093EF0263
:1035D0006091EE0284E090E00E9471356C2F82E2EF
:1035E00090E00E94713582E00E94BE1A80912F0304
:1035F00080FF0CC01F92DF938BED92E09F938F931F
:103600000E9427070F900F900F900F90DF91CF919E
:10361000089521E030E001C0220F8A95EAF78091F9
:10362000E603822B0E94A01A0895809394020E94C0
:10363000931A089510929202E2E2F2E086E0DF012E
:103640001D928A95E9F70E94931A0895AAE2B0E0C4
:10365000ECE2FBE10C9466348BED93E02091F100F9
:10366000DC012D93CD01B3E0833E9B07B9F7809138
:10367000DC03833009F472C0B8F4813009F449C026
:10368000823009F4B3C08091E80083FF91C2809139
:10369000DB039091DC039A3008F08AC2E92FF0E056
:1036A000E65FF94C0C94C2348A3009F48EC08B303A
:1036B00009F471C0893039F78091DB03813219F741
:1036C0008091DF039091E003009711F00297D9F603
:1036D0008091E800877F8093E8008091E80082FF76
:1036E00038C09091F3008091F200029731F48091FC
:1036F000F100813011F0863021F48091F100809347
:10370000CE038091E8008B778093E8000E94AA079F
:10371000BACF8091DB03813A09F0B5CF8091E80000
:10372000877F8093E8008091DF039091E003892BED
:1037300061F468E08FEC93E070E00E94560880919D
:10374000E8008B778093E8009ECF60E090E080E017
:10375000F3CF8091D9038111C0CF95CF8091DB0346
:10376000813A09F090CF8091DF039091E003892B9B
:1037700009F089CF8091E800877F8093E8008091ED
:10378000E80080FFFCCF809164018093F10080917C
:10379000E8008E77B9CF8091DB03813209F073CFD7
:1037A0008091DF039091E003892B09F06CCF809129
:1037B000E800877F8093E8000E94AA078091DD03DC
:1037C000809364010E941A1B5ECF8091DB038132DB
:1037D00009F059CF8091E800877F8093E8000E942C
:1037E000AA078091DE038093CD034DCF8091DB0348
:1037F000813A09F048CF8091E800877F8093E80004
:103800008091E80080FFFCCF8091CD03BECF80384F
:1038100099F0823809F0CCC18091DF038F70873036
:1038200008F0C6C18093E9008091EB0085FB8827F2
:1038300080F91092E90006C08091D7039091D803D7
:10384000911182609091E800977F9093E8008093B7
:10385000F1001092F1008091E8008E77A5C18823D5
:1038600009F493C1823009F0A3C18091DD03811175
:1038700096C18091DF038F702FEF280F263008F05C
:1038800097C18093E9002091EB0020FF88C193301D
:1038900031F48091EB0080628093EB0080C19091C5
:1038A000EB0090619093EB0021E030E001C0220F2B
:1038B0008A95EAF72093EA001092EA008091EB00E3
:1038C0008860EACF811174C11091DD031F77809168
:1038D000E3008078812B8093E3008091E800877F6C
:1038E0008093E8000E94AA078091E80080FFFCCF47
:1038F0008091E30080688093E30082E0111183E00F
:103900008093D90355C18058823008F051C120916D
:10391000DD033091DE032C3DE3E03E07A1F583E0BB
:103920008A838AE289834FB7F894DE01139620E0F8
:103930003EE051E2E32FF0E050935700E49120FF86
:1039400003C0E295EF703F5FEF708E2F90E0EA309A
:10395000C0F0C7968D939D932F5F243159F74FBFC9
:103960008091E800877F8093E8006AE270E0CE01F2
:1039700001960E9456088091E8008B778093E800BA
:1039800017C1C096E7CF8091DF039091E003432FEA
:1039900055274330510509F44AC078F541305105A7
:1039A00009F47AC08BE790E0EBECFBE04230510584
:1039B00009F0FEC02091E800277F2093E8002091C5
:1039C000E1033091E2038217930708F49C0140E081
:1039D0002115310509F065C0411163C08091E800EF
:1039E00082FDC9CF8091D903882329F2853019F24D
:1039F0008091E80083FFF2CFBECF4132510509F438
:103A00003CC04232510509F0D3C08430910508F022
:103A1000CFC0FC01EE0FFF1FE25FFD4F0190F08170
:103A2000E02D865F9D4FDC018C9190E01AC033271A
:103A300021303105D1F02115310561F022303105F9
:103A400009F0B6C0E8E5FCE0E4918E2F90E0E8E5EF
:103A5000FCE007C0ECE8FCE0E4918E2F90E0ECE89D
:103A6000FCE0009709F4A4C0A5CFECE7FCE0E491EA
:103A70008E2F90E0ECE7FCE0F4CF8430910508F065
:103A800097C0880F991FFC01EA5EFD4F0190F081FD
:103A9000E02D89E090E08ECF82E190E0E6E4FCE06A
:103AA00089CF8091D903882309F465CF853009F443
:103AB00062CF8091E80083FD5ECF8091E80082FDB7
:103AC0008DCF8091E80080FF83CF9091F3008091AB
:103AD000F2002115310519F08830910550F041E0D0
:103AE000089709F040E08091E8008E778093E80025
:103AF0006FCF44914093F1003196215031090196E6
:103B0000E8CF803809F054C08091E800877F809327
:103B1000E8008091DA038093F1009DCE811148C0C6
:103B20001091DD03123008F043C08091E800877FD8
:103B30008093E8001093DA030E94AA07112311F082
:103B400084E005C08091E30087FDFACF81E0809397
:103B5000D90342E061EC81E00E94C90742E261ECD6
:103B600084E00E94C90742E261EC82E00E94C9073A
:103B700042E260EC83E00E94C90742E261EC85E02A
:103B80000E94C9078091D90313C08091DD03813061
:103B900079F481E0933009F080E08093D8031092AB
:103BA000E9008091E800877F8093E8000E94AA07DF
:103BB0008091E80083FF0AC08091E800877F8093AE
:103BC000E8008091EB0080628093EB00AA96E3E02E
:103BD0000C9482340E941A1B2FEF84E39CE0215046
:103BE00080409040E1F700C0000088E19CE00FB603
:103BF000F894A895809360000FBE90936000FFCF6B
:103C0000882321F00E94B10B0E94211A0895882375
:103C100039F090919202982B909392020E94211A6F
:103C20000895882309F44DC0823879F40E94AC10BD
:103C300081FF47C089E30E94C50B0E94211A89E3D6
:103C40000E94B80B0E94211A0895833859F40E94EB
:103C5000AC1080FF36C083E50E94C50B0E94211A7C
:103C600083E5EECF843859F40E94AC1082FF29C05E
:103C700087E40E94C50B0E94211A87E4E1CF9CEFE4
:103C8000980F913AE8F290E2980F983050F48770CC
:103C900091E001C0990F8A95EAF7892F0E94B10B34
:103CA000D1CF9BE5980F933028F490E080E00E94FC
:103CB000F7080895885A873120F490E080E00E9448
:103CC000E1080895CF93C82F8823C9F08238C9F43A
:103CD0000E94AC1081FD13C089E30E94C50B0E94B5
:103CE000211A2FEF87EE93E0215080409040E1F7BA
:103CF00000C0000089E30E94B80B0E94211ACF91F6
:103D000008958338A1F40E94AC1080FDF8CF83E5BC
:103D10000E94C50B0E94211A2FEF81EE94E02150E2
:103D200080409040E1F700C0000083E5E4CF843894
:103D3000A1F40E94AC1082FDE2CF87E40E94C50B83
:103D40000E94211A2FEF81EE94E021508040904094
:103D5000E1F700C0000087E4CECF8CEF8C0F813AF2
:103D600068F4E2E2F2E08191C817A1F122E0E832C2
:103D7000F207C9F78C2F0E94C50BBFCF80E28C0FD2
:103D8000883068F4C77021E030E001C0220FCA9586
:103D9000EAF780919202822B80939202AECFEBE5FC
:103DA000EC0FE33040F4F0E0E456FE4F808190E009
:103DB0000E94F708A4CFC85AC73108F0A0CFEC2F53
:103DC000F0E0EE0FFF1FE156FE4F808191810E94CF
:103DD000E10895CF8C2F0E94B80B0E94211ACACF00
:103DE0001F93CF93DF93182FD0E0C0E0893311F4F5
:103DF000C0E5D0E0812F0E94621E209739F4812F08
:103E00000E94111EDF91CF911F9108958FE99FE0CD
:103E10000197F1F700C000002197EFCF0F931F9398
:103E2000CF93DF93C62FD42F022FFC0182818823EA
:103E3000A9F06093E5030E94D5089093E403809372
:103E4000E303C77081E001C0880FCA95EAF70E94BA
:103E5000071EDF91CF911F910F9108958091E50387
:103E6000681332C08091E3039091E4030E94BA0882
:103E7000883C910548F510E21D0FCD17B9F080E29E
